:1000000088C0F8C1A1C0A0C09FC09EC09DC09CC0B8
:100010009BC09AC099C098C097C096C095C094C024
:1000200093C092C091C004030904180372006100D8
:10003000700068006E00650074002E006E006500A0
:1000400074000A033100300030003000050109045B
:10005000A1010901A100850109300931150026FF20
:100060000075089502810205091901290815002566
:1000700001750195088102C0C005010904A10109AB
:1000800001A100850209300931150026FF0075081D
:10009000950281020509190129081500250175013C
:1000A00095088102C0C005010904A1010901A10050
:1000B000850309300931150026FF00750895028176
:1000C0000205091901290815002501750195088106
:1000D00002C0C005010904A1010901A100850409AC
:1000E000300931150026FF007508950281020509C7
:1000F0001901290815002501750195088102C0C064
:10010000120101010000000881179D0A020101028D
:10011000030111241FBECFE5D4E0DEBFCDBF10E048
:10012000A0E6B0E0E4E0FEE002C005900D92AC3A3B
:10013000B107D9F711E0ACEAB0E001C01D92A231DD
:10014000B107E1F739D35CC65BCF85B7836085BF64
:100150008BB780648BBF83EC8093E80008950F9386
:100160001F93CF93DF939091F80019160CF0A6C05F
:100170002091F5008091F4008D3209F095C08AE558
:10018000809361009B3009F08FC0CCE0D0E0C21BAF
:10019000D109C450DF4F8881807609F077C0109272
:1001A000E6008981882351F41092E70086EE90E002
:1001B0009093F7008093F60032E06BC0853021F415
:1001C0008A818093F90060C0863009F043C08B813A
:1001D0008130E1F1823019F4CE016FD259C0833001
:1001E00049F58A81882341F486E290E09093F700F4
:1001F0008093F60034E050C0813041F48AE290E010
:100200009093F7008093F60038E146C0823041F4C5
:1002100083E690E09093F7008093F60036E139C0D2
:100220008330C9F582E490E09093F7008093F60064
:100230003CE032C0813241F48FEB90E09093F700C4
:100240008093F60039E028C0823229F5CE0135D2FC
:10025000382F22C0883019F48BEF90E00AC0893023
:1002600021F48A818093FB000FC08A3041F486EE2E
:1002700090E09093F7008093F60031E00AC08B3055
:1002800019F483EC8093E80030E003C0CE0143D240
:10029000382F20E802C030E020EC8F81882339F429
:1002A0008E81831728F003C080E020E801C0832FEF
:1002B0002093AC00809360001092F8008091610060
:1002C00084FF49C0809160008F3F09F444C0182F1B
:1002D000893008F018E0811B809360008091AC00A9
:1002E00080FD02C00BE401C003EC8F5F8093AC0083
:1002F0002091F6003091F70086FD05C0D901912FBD
:10030000EEEDF0E011C0AEEDB0E080E090E006C0B0
:10031000F901E80FF91FE491ED9301961817C1F761
:1003200005C08D91819391509923D9F7F901E10F7F
:10033000F11DF093F700E093F6008EED90E0612F51
:1003400055D0183019F08FEF809360000093DD00D6
:100350001C5F109361009AE080B3857031F4915076
:10036000D9F71092F9001092F300DF91CF911F910D
:100370000F9108951F93DC01162F8091620084FF76
:100380000AC08091E80098E889278093E800912FBF
:10039000E9EEF0E007C08AE580936200F8CF8D9126
:1003A000819391509923D9F789EE90E0612F1ED067
:1003B0001C5F109362001F910895A82FB92F8FEF33
:1003C0009FEF41E050EA615070F02D9138E0722FBC
:1003D000782796958795269570FF02C084279527E4
:1003E0003A95A9F7F0CF809590950895E6DF8D9323
:1003F0009D930895CF93CFB7CF93809BFECF809BE3
:1004000009C0809B07C0809B05C0809B03C0809B68
:1004100001C09EC0DF93C091F500DD27C450DF4FBF
:10042000809B02C0DF91EBCF2F930F931F9300B3FC
:100430002FEF00FB20F94F933F9310B34FEF0127AD
:1004400000FB21F93BE031C04E7F012F10B321604A
:1004500028C0102F4D7F2260000000B329C04B7FC1
:100460002460012F000010B32BC010B3477F286019
:100470002AC04F7E00B320612CC04F7D10B3206294
:100480002FC04F7B00B3206432C0422700B3499392
:100490004FEF0000102710FB20F910B31570A9F1E1
:1004A000297F91F2012700FB21F900B3237F89F214
:1004B0003150F0F1102710FB22F910B3277E79F2AA
:1004C000012700FB23F92F7C81F200B3102710FBDA
:1004D00024F92F7971F200C010B3012700FB25F930
:1004E0002F7359F200C000B3102710FB26F92230F9
:1004F00040F200C010B3012700FB27F9243028F692
:100500004F77206810B30000F9CF3B50319533305E
:1005100010E41ABFB8F0C31BD0400881033C41F17E
:100520000B3431F11981412F1F772091F3001217FD
:1005300031F4093691F10D3279F0013E69F022274C
:100540002093FA003F914F911F910F912F91DF91CE
:10055000CF91CFBFCF9118950093FA003F914F9163
:100560001F910F912F91DF91CAB7C6FD46CFF0CFF3
:100570000091FA00002331F31091F8001123A1F546
:100580003430A2F13093F8000093F4001091F5009C
:100590003BE0311B3093F50029C00091F800013099
:1005A0001CF50AE547FD09C03091610034FD20C00B
:1005B00000936100CDEDD0E01FC03091620034FDAA
:1005C00017C000936200C8EED0E016C0052710E007
:1005D00002BB1FC0052722C0052727C005272CC046
:1005E000052710E002BB33C04AE503C042ED01C05D
:1005F000432FC4E1D0E032E011B31560909A02B30A
:1006000011BB5F9355E020E820FF052702BB27952B
:1006100017951C3FD8F620FF0527279502BB179595
:100620001C3FC0F620FF05272795179502BB1C3FEE
:1006300098F620FF0527279517951C3F02BB70F6FB
:1006400000C0499120FF052702BB279517951C3F45
:1006500038F620FF0527279502BB17951C3F38F574
:1006600020FF05272795179502BB1C3F10F520FF9B
:100670000527279517951C3F02BBE8F4242F3A95D0
:1006800019F60A7F5F9102BB00C01091F900C651B4
:10069000D04011F01093F30010E41ABF016011B3C1
:1006A0001A7F402F4A7F02BB11BB42BB4BCF0527AD
:1006B000D3CF0527D8CF0527DDCFFC0180818076F9
:1006C00041F58181863029F583818230D1F08232F3
:1006D00069F08130F1F48091B1009091B200909373
:1006E000F7008093F6008091B30008958091AE00EA
:1006F0009091AF009093F7008093F6008091B00046
:10070000089587E790E09093F7008093F60082E2E7
:10071000089580E00895DC0127EB30E03093F70086
:100720002093F6008C918076803209F043C01196B8
:100730008C911197823091F08A3001F18130D1F59E
:100740001092B400E091B500F091B6000784F089F2
:10075000E02DC90112966C910995089512969C910D
:10076000892F8150883030F5892F90E08E539F4F2C
:100770009093F7008093F60081E008951296EC9133
:100780001297EE2359F4E3ECF0E013968C91139753
:10079000819380E0EB3CF807C1F70CC08E2F8150AD
:1007A000883040F4F0E0EE53FF4F13968C91808335
:1007B00080E0089580E008958F929F92AF92BF925B
:1007C000CF92DF92EF92FF920F931F93DF93CF931D
:1007D000CDB7DEB728970FB6F894DEBF0FBECDBFFA
:1007E000FE01319688E0DF011D928A95E9F7B89AFB
:1007F00087B3897F87BB88B3866088BBC09880E356
:1008000095E70197F1F786B390E086709070959523
:100810008795823009F4E6D019D2FC019093B60096
:100820008093B500838194819093AF008093AE0054
:1008300081818093B00087819085009731F09093FB
:10084000B2008093B100858107C080E091E0909371
:10085000B2008093B100C4D28093B3008091B00005
:100860008093900014BA8FEF85BB88EF82BB85E040
:1008700081BB11BA83BF8FE085BD84EC83BDE0915D
:10088000B500F091B6000184F285E02D09955DDC9C
:10089000E091B500F091B6000384F485E02D099550
:1008A000789490E8892E81E0C82ED12C99249394D5
:1008B0005E010894A11CB11CA89551DC08B607FC88
:1008C00002C0FF242AC088BEE091B500F091B600B6
:1008D0000384F485E02D0995FF2400E010E012C0A8
:1008E0000584F685E02D802F8F5F0995882341F0E0
:1008F000C601002E02C0880F991F0A94E2F7F82A59
:100900000F5F1F4FE091B500F091B60080819927ED
:1009100087FD9095081719071CF308B600FE29C03B
:1009200098BE4091B5005091B600D50120E030E06E
:1009300018C0F901ED53FF4FE081EE2379F08C915F
:10094000853018F085508C9309C0EC93C601022EB7
:1009500002C0880F991F0A94E2F7F82A2F5F3F4FD1
:100960001196FA018081992787FD909528173907FC
:1009700004F3FF2009F4A0CF00E010E0EF2CFF24E7
:10098000E7FCF09422C0C701002E02C09595879520
:100990000A94E2F780FF17C08091620084FF13C0C1
:1009A000602F6F5F0784F089E02D87EB90E0099559
:1009B000682F87EB90E0DEDC02C0D1DBA895809148
:1009C000620084FFFACF0F5F1F4FE091B500F091F6
:1009D000B6008081992787FD9095081719070CF0BC
:1009E0006BCFD1CF1092AA000895AC9A80E38A957C
:1009F000F1F7AC988091CB00882309F448C020E03F
:100A000030E070E060E098E1892F8A95F1F7AD98C9
:100A1000770F660F9B9B71609A9B6160892F8A9507
:100A2000F1F7AD9A2F5F3F4F2830310569F720E08D
:100A300030E050E040E098E1892F8A95F1F7AD98D9
:100A4000550F440F9B9B51609A9B4160892F8A955B
:100A5000F1F7AD9A2F5F3F4F2830310569F780E0FD
:100A600090E038E1232F2A95F1F7AD98232F2A95AE
:100A7000F1F7AD9A019688309105A1F77093CD00FA
:100A80006093CE005093CF004093D000089520E0B3
:100A900030E090E040E050E060E078E1872F8A9518
:100AA000F1F7AD98990F440F550F660F9B9B91601E
:100AB0009A9B4160999B5160989B6160872F8A95B2
:100AC000F1F7AD9A2F5F3F4F2830310539F79093FA
:100AD000CD004093CF005093D1006093D30020E02D
:100AE00030E078E1872F8A95F1F7AD989695469595
:100AF000569566959B9B90689A9B4068999B506819
:100B0000989B6068872F8A95F1F7AD9A2F5F3F4FCA
:100B10002830310539F78091AA00882321F180918E
:100B2000CC009F3F11F4816001C08E7F8093CC0088
:100B30008091CC004F3F11F4826001C08D7F809383
:100B4000CC008091CC005F3F11F4846001C08B7FAA
:100B50008093CC008091CC006F3F11F4886001C07D
:100B6000877F8093CC008091CC0080FD90E09093B3
:100B7000CE0081FD40E04093D00082FD50E05093D4
:100B8000D20083FD60E06093D40008951F931FB7E7
:100B9000F894A49AA59A84B3807F84BB85B38F60B0
:100BA00085BBAD9AAC981092CC001FDF8091AA0053
:100BB000882321F58091CE008F3F29F48091CC00CD
:100BC00081608093CC008091D0008F3F29F4809188
:100BD000CC0082608093CC008091D2008F3F29F4BA
:100BE0008091CC0084608093CC008091D4008F3FB2
:100BF00029F48091CC0088608093CC00AC9A80E38B
:100C00008A95F1F7AC9880E090E030E040E058E160
:100C1000252F2A95F1F7AD989B9905C08331910551
:100C200019F441E001C03F5F252F2A95F1F7AD9AF5
:100C300001968831910561F7442329F0373119F481
:100C400081E08093CB001FBF1F9108958CE490E05A
:100C500090939D0080939C0089E990E00895CF9344
:100C6000DF93EC01653010F080E094C08091CB0000
:100C7000E62FFF27E7FDF095882359F1DF01119753
:100C80002097F9F06883FD01E353FF4F808180FDD9
:100C900002C090E801C09FEF81FD90E09983FD01C3
:100CA000E353FF4F808182FD02C090E801C09FEFB7
:100CB00083FD90E09A83FD01E353FF4F8081807FA5
:100CC0008B83FD01E353FF4F8081AB52BF4F8C9369
:100CD00060C0DF011197209709F44FC06883BD0100
:100CE000660F771FFB01E353FF4F808180FD02C039
:100CF00090E801C09FEF81FD90E09983FB01E353F1
:100D0000FF4F808182FD02C090E801C09FEF83FD0C
:100D100090E09A838091CC0090E00A2E02C09595D5
:100D200087950A94E2F7FB01E353FF4F80FF03C06E
:100D30008081807F21C06081462F50E09A0120741D
:100D4000307075E0359527957A95E1F7CA01807284
:100D5000907033E0959587953A95E1F7282B661FBB
:100D60006627661F262B4071507055954795242B9A
:100D700081818295807F822B8B83FD01EE0FFF1F87
:100D8000DF01A353BF4F8D919C91EB52FF4F918395
:100D9000808384E0DF91CF91089581509091CB00C2
:100DA000A82FBB27A7FDB095992361F020E0FD0196
:100DB000EB52FF4FA353BF4F9C918081981771F066
:100DC00021E00CC0BD01660F771FCB0183539F4FFD
:100DD0006B527F4F42E050E006D0282F822F0895BB
:100DE00082E190E00895FB01DC0104C08D91019047
:100DF000801921F441505040C8F7881B990B089581
:040E0000F894FFCF94
:100E0400FF5A5A140334006E0065007300340073F3
:100E1400006E006500730009022200010100803C9D
:100E2400090400000103000000092101010001225E
:100E340000000705810308000A04B4000000000054
:0C0E44000000C605F504CD062F060100D5
:00000001FF
